:10036600403E3B352D23180C403518F3D2C1C4DC72
:100376004023E7C1D20C3B35400CC4DC2D35E7C128
:1003860040F3C4232DCAE73E40DCE73ED2F33BCA26
:1003960040CA180CD23EC42340C13BCA2DDC18F318
:1003A600645A504600000000640000003C00000053
:1003B600640000003C000000640000463C000000B1
:1003C600640000003C0000006400000000320000F1
:1003D6006400000000320000645A50463C320000BF
:0303620001082D62
:0A000300EF60047F408002AF082286
:10000D008F0B8D0C8B0D8A0E890F751300751200D9
:10001D00751100751000E4F514E4F515E51475F08F
:10002D0008A4AB0D250FF9E50E35F0FA7E00E92594
:10003D0015F9EE3AFA120472FF3395E0FEAD0BEDB1
:10004D003395E0FCE51475F008A42466F582E434DC
:10005D0003F583E5822DF582EC3583F583E493FD7D
:10006D003395E0FC12048BAD0CED3395E0FCE515FA
:10007D0075F008A42466F582E43403F583E5822D3A
:10008D00F582EC3583F583E493FD3395E0FC1204A2
:10009D008BEF780CCEA2E713CE13D8F8FFEE339585
:1000AD00E0FDFCE5132FF513E5123EF512E5113DCC
:1000BD00F511E5103CF5100515E515640860030212
:1000CD0000290514E51464086003020026AF0B1225
:1000DD000003E4FCFDFEAB13AA12A911A810120433
:1000ED009FA804A905AA06AB07AF0C120003E4FCF8
:1000FD00FDFE12049F780E1204EEEE3395E0FDFC2A
:01010D0022CF
:10010E00E4F509E4F50AAF09AD0A7BFF7A0379A697
:10011E0012000DE509C43354E02408F582E43401DD
:10012E00F58375F004E50A12053F120502050AE58E
:10013E000AC3940840D00509E509C3940840C422B7
:10014E0090000012050E0000000090000412050E33
:10015E0000000000E4F509E4F50A90000012050E17
:10016E0000000000E4F50BE4F50C900000E0F8A3AD
:10017E00E0F9A3E0FAA3E0FBC000C001C002C00397
:10018E00AF0C120003AE07AF0B120003EF8EF0A4FC
:10019E00FFAEF0E4FCFDC004C005C006C007AF0C06
:1001AE00EF3395E0FEEF7802C333CE33CED8F9FDB0
:1001BE00AC06AF0BEF3395E0FEEF7805C333CE33CD
:1001CE00CED8F92408F582EE3401F583E5822DF5BB
:1001DE0082EC3583F583E0F8A3E0F9A3E0FAA3E01F
:1001EE00FBD007D006D005D00412049FC004C00572
:1001FE00C006C007AF09EF3395E0FEEF7803C333B7
:10020E00CE33CED8F92466F582EE3403F583AF0BE8
:10021E00EF3395E0FEE5822FF582EE3583F583E42C
:10022E0093FF3395E0FEFDFCD003D002D001D00049
:10023E0012049FC004C005C006C007AF0AEF339575
:10024E00E0FEEF7803C333CE33CED8F92466F582C1
:10025E00EE3403F583AF0CEF3395E0FEE5822FF518
:10026E0082EE3583F583E493FF3395E0FEFDFCD0FB
:10027E0003D002D001D00012049F78181204EED0E1
:10028E0003D002D001D000EB2FFFEA3EFEE93DFD88
:10029E00E83CFC900000120502050CC3E50C6480DE
:1002AE0094885003020178050BC3E50B6480948893
:1002BE005003020175900000E0FCA3E0FDA3E0FEF8
:1002CE00A3E0FF78021204EE9000041205029000E3
:1002DE0004E0FCA3E0FDA3E0FEA3E0FFC004C00524
:1002EE00C006C007AF0AEF3395E0FEEF7802C333C6
:1002FE00CE33CED8F9FDAC06AF09EF3395E0FEEF65
:10030E007805C333CE33CED8F92408F582EE340007
:10031E00F583E5822DF582EC3583F583D007D00683
:10032E00D005D004120502050AC3E50A648094883C
:10033E0050030201680509C3E509648094885003DF
:04034E000201652221
:1003520075900112010E75900212014E75900322E2
:030000000203E612
:0C03E600787FE4F6D8FD75811502042D27
:10047200BB010689828A83E0225002E722BBFE0288
:09048200E32289828A83E49322BB
:10048B00EFF88DF0A4FFEDC5F0CEA42EFEEC88F0B6
:04049B00A42EFE226B
:10049F00E88FF0A4CC8BF0A42CFCE98EF0A42CFCFC
:1004AF008AF0EDA42CFCEA8EF0A4CDA8F08BF0A47A
:1004BF002DCC3825F0FDE98FF0A42CCD35F0FCEBD9
:1004CF008EF0A4FEA9F0EB8FF0A4CFC5F02ECD399E
:0F04DF00FEE43CFCEAA42DCE35F0FDE43CFC220B
:1004EE00E86010ECA2E713FCED13FDEE13FEEF1324
:0404FE00FFD8F02211
:0C050200ECF0A3EDF0A3EEF0A3EFF0226C
:10050E00A8828583F0D083D082120525120525128C
:10051E000525120525E473E493A3C583C5F0C583B1
:10052E00C8C582C8F0A3C583C5F0C583C8C582C837
:01053E00229A
:0C053F00A42582F582E5F03583F58322C7
:1003F200020352E493A3F8E493A34003F68001F2CC
:1004020008DFF48029E493A3F85407240CC8C3330B
:10041200C4540F4420C8834004F456800146F6DFDA
:10042200E4800B0102040810204080900362E47E05
:10043200019360BCA3FF543F30E509541FFEE493CF
:10044200A360010ECF54C025E060A840B8E493A396
:10045200FAE493A3F8E493A3C8C582C8CAC583CAC1
:10046200F0A3C8C582C8CAC583CADFE9DEE780BE79
:010365000097
:00000001FF
